:100000008A110A1205280000090083168101831253
:100010008B0183168C01831207309F0083162330D7
:1000200085003F30860083122C14AC142C15AC15BF
:100030002C16B301B40186179030A0000130A10046
:100040005E2186132C30A0000130A1005E218617AE
:100050009030A0000130A1005E21861306182C14F8
:10006000061C2C102C184D2886173308013EB300AF
:1000700034080318013E003EB400F430A000013003
:10008000A1005E218613F430A0000130A1005E21A2
:1000900006182C14061C2C1032281F3083058618D5
:1000A000AC14861CAC10AC186E2886173308053EBD
:1000B000B30034080318013E003EB400F430A00041
:1000C0000130A1005E218613F430A0000130A100B0
:1000D0005E218618AC14861CAC1053281F30830593
:1000E00006192C15061D2C112C198F28861733087C
:1000F0000A3EB30034080318013E003EB400F43059
:10010000A0000130A1005E218613F430A000013070
:10011000A1005E2106192C15061D2C1174281F3014
:1001200083058619AC15861DAC11AC19B02886174D
:1001300033081E3EB30034080318013E003EB400ED
:10014000F430A0000130A1005E218613F430A0003D
:100150000130A1005E218619AC15861DAC119528D1
:100160001F308305061A2C16061E2C122C1AD128B5
:10017000861733083C3EB30034080318013E003EA6
:10018000B400F430A0000130A1005E218613F430E9
:10019000A0000130A1005E21061A2C16061E2C12AA
:1001A000B6281F308305861A372986130617C830EC
:1001B000A000A1015E2106130130AD00AE012D08A3
:1001C000A0002E08A1003408A30033084B21031D12
:1001D00004290130AF002F083C3C031CF828E8300C
:1001E000A0000330A1005E210130AF07031CEB2803
:1001F0001F3083050130AD0700300318013E03189E
:100200000429AE07031CDF281F3083050130B0002E
:100210003008053C031C1C2906172C30A0000130B7
:10022000A1005E210613E830A0000330A1005E218A
:100230000130B007031C08291F3083050130B000CE
:100240003008053C031C342906175830A000023042
:10025000A1005E210613E830A0000330A1005E215A
:100260000130B007031C20291F30830586171F307B
:1002700083052E283A293B29A20005304E29A200E9
:1002800002304E29A20006304E29A20003304E292A
:10029000A20004304E29A20001304E29A8002308F4
:1002A0002102031D552922082002043003180130C1
:1002B000031902302805031DFF300800A0080319A8
:1002C00069297021A0030000000000000000000068
:1002D0005E29A108031908007021A103A0035E296B
:1002E0000C30A500A50B7229000000001230A200FE
:1002F000A20B7F29812181210000000008008121BB
:0E03000078290D30A400A40B8329000008000A
:02400E00313F40
:00000001FF
